:0200000480007A
:100000006F00C0006F20C02B6F20802B930000007A
:10001000130100009301000013020000930200008E
:100020001303000093030000130400009304000076
:10003000130500009305000013060000930600005E
:100040001307000093070000130800009308000046
:100050001309000093090000130A0000930A00002E
:10006000130B0000930B0000130C0000930C000016
:10007000130D0000930D0000130E0000930E0000FE
:10008000130F0000930F00009702000093820201FB
:10009000739052307350447497020000938202F7B9
:1000A0007390523017E100001301C1E3F32240F1D5
:1000B0009392C2003301510073100134EF20D0132A
:1000C000173500001305C5946F20407383328510E7
:1000D000739012148330850003310501833185014B
:1000E000033205028332850203330503833385031C
:1000F00003340504833485048335850503360506FA
:1001000083368506033705078337850703380508D7
:10011000833885080339050983398509033A050AB7
:10012000833A850A033B050B833B850B033C050C97
:10013000833C850C033D050D833D850D033E050E77
:10014000833E850E033F050F833F850F033505056D
:10015000730020107311011423341100233C31006B
:10016000233041022334510223386102233C7102BF
:1001700023308104233491042338A104233CB104A7
:100180002330C1062334D1062338E106233CF1068F
:10019000233001092334110923382109233C310973
:1001A0002330410B2334510B2338610B233C710B5B
:1001B0002330810D2334910D2338A10D233CB10D43
:1001C0002330C10F2334D10F2338E10F233CF10F2B
:1001D000F312011423385100F32200102330511080
:1001E000F322101423345110F32230142338511009
:1001F000F3222014233C5110130501006F20C03757
:1010000000000000000000000000000000000000E0
:1010100000000000000000000000000000000000D0
:1010200000000000000000000000000000000000C0
:1010300000000000000000000000000000000000B0
:081040000000000000000000A8
:10200000B367B500B3E7C70093F77700B306C50021
:10201000638407023386C50093070500637ED502FB
:1020200003C705009385150093871700A38FE7FE6C
:10203000E398C5FE67800000E37ED5FE93070500A8
:1020400003B70500938787009385850023BCE7FECF
:10205000E3E8D7FE6780000067800000130101FFFE
:10206000B367C500233081002334110093F7770054
:10207000130405003307C500638207026376E50099
:1020800093F5F50FEFF09FFD8330810013050400F9
:1020900003340100130101016780000093F5F50F7F
:1020A0009717000083B7870EB385F502E37EE5FC42
:1020B000930705009387870023BCB7FEE3ECE7FE98
:1020C0008330810013050400033401001301010172
:1020D0006780000083470500638E070093070500B3
:1020E00003C7170093871700E31C07FE3385A7403B
:1020F000678000001305000067800000834705002B
:10210000938515001305150003C7F5FF638A0700C3
:10211000E386E7FE1B8507003B05E540678000007E
:10212000130500006FF05FFFB367B50093F777000A
:10213000639E0702137886FF330805016378050361
:10214000930705006F000001938787009385850042
:1021500063F8070183B6070003B70500E386E6FED0
:102160003385A7403306A640138507003386C50094
:102170006F00400103C705008347F5FF93851500F5
:10218000639AE70013051500E396C5FE13050000EA
:10219000678000003B85E7406780000093070500EB
:1021A00003C705009387170093851500A38FE7FEEB
:1021B000E31807FE6780000003470500930600024E
:1021C000930705006318D70003C71700938717000C
:1021D000E30CD7FE9306D0026300D7069306B00245
:1021E0006300D70483C607009305000063820604DA
:1021F0001305000093871700131725001B8606FDA3
:1022000083C607003307A700131717003305E6003E
:10221000E39206FE638005023305A040678000005C
:1022200083C617009305000093871700E39206FC0E
:10223000130500006780000083C617009305100097
:1022400093871700E39606FA130500006FF09FFED0
:1022500083470500638007049305101017F7FFFFFD
:10226000130747DA93950503033607001305150096
:10227000B3E6B700630A060097F7FFFF23B407DC55
:1022800083370700E39A07FE2330D7008347050012
:10229000E39C07FC6780000017F7FFFF130787D652
:1022A00083370700638A070097F7FFFF23BC07D82F
:1022B00083370700E39A07FE2330A7006F00000072
:1022C000130101FF1305903423341100EFF0DFFCFC
:1022D000130101FE1306810093077101130890009A
:1022E0006F008000930707009376F50013870600C0
:1022F000930500036374D800930570053B07B7008E
:102300002380E700135545001387F7FFE31CF6FC15
:1023100083478100230C010063820704130510101A
:102320009306060017F7FFFF1307C7CD1315050324
:10233000833507009386160033E6A700638A0500FD
:1023400097F7FFFF23B007D083370700E39A07FE14
:1023500083C706002330C700E39C07FC130101027A
:1023600067800000130101FB9307100037F7FFFFA0
:102370002322F1002334110423308104233C9102F1
:10238000233821032334310323304103233C5101FB
:1023900023340100B306E500B7E7030063F6F6183F
:1023A0009359C5009384096017490000130989C532
:1023B00093973400B307F90083B707003374E5003F
:1023C0006396071017870000130747C4033A0700F6
:1023D00063000A1883378A009786000083B686C296
:1023E0002330F700638CD712130641009305810058
:1023F00013050400833A0A00EF00C0606310051063
:1024000093D6CA009396A60093E6F60193973400FC
:10241000B307F90013E7060C23B0E70073000412BA
:1024200097370000938707BE93994900B387370118
:1024300003B707006318071203370A00B705040043
:1024400023B0E70003378A0023B4E700F3A50510A3
:10245000B707E0FFB307F4003716000013070400C6
:102460003386C70003B3070083B8870003B80701AA
:1024700003B5870123306700233417012338070190
:10248000233CA7009387070213070702E39CC7FCBE
:102490007390051093973400B304F90023B0D4006F
:1024A000730004120F100000833081040334010410
:1024B000833481030339010383398102033A010222
:1024C000833A8101130101056780000013F70704B7
:1024D0006302070413F70708631207061307F000E7
:1024E00093E70708639CE50493943400B3049900D0
:1024F00023B0F400730004126FF01FFB83360A0050
:102500008337810093D6C6009396A600B3E6F60003
:102510006FF0DFEF93E707046FF01FFD9787000070
:1025200023B207AE6FF05FEC17150000130585C6E8
:10253000EFF01FD213053000EFF01FD61715000083
:102540001305C5C9EFF0DFD013053000EFF0DFD47D
:1025500017150000130505CDEFF09FCF13053000D0
:10256000EFF09FD317150000130545CDEFF05FCEB8
:1025700013053000EFF05FD2130101F82338810614
:10258000233C11062334910623302107233C3105D7
:10259000233841052334510523306105233C710361
:1025A00023388103233491032330A103233CB10159
:1025B00013040500EF0080446312050E8335841177
:1025C000930780006380F510930720006380F50671
:1025D000938745FF130710006376F7009307F00019
:1025E000639CF51E03350411EFF0DFD713050400DB
:1025F00003340107833081078334810603390106E0
:1026000083398105033A0105833A8104033B0104C0
:10261000833B8103033C0103833C8102033D0102B0
:10262000833D8101130101086FD05FAA0337841035
:1026300093773700639E0706EF0780007310300022
:102640000327070083A707006300F7061305101090
:102650009307100497160000938646C217F7FFFFF2
:102660001307479A13150503833507009386160051
:1026700033E6A700638A050097F7FFFF23B4079CA2
:1026800083370700E39A07FE83C706002330C7009D
:10269000E39C07FC13053000EFF01FC01305040096
:1026A000EFD0DFA26FF09FF113051000EFF0DFBE57
:1026B00017150000130585C6EFF09FB9130530000C
:1026C000EFF09FBD83270405B7140000973A000080
:1026D000938A4A932334F100174D0000130D8D9215
:1026E000B70C0400370CE0FF178A0000130A8A9128
:1026F000978B0000938B8B9137FB030093D7C4001B
:102700001399470033872A0103370700630C070832
:102710009387076093973700B307FD0083B90700DD
:1027200093F709046380070AF3AD0C103384840126
:10273000371600009305040013850400EFF0DF9EB8
:102740006304050493F909086380090AB7160000B9
:102750001387040093070400B386D40003380700EE
:1027600003358700833507010336870123B007014E
:1027700023B4A70023B8B70023BCC7001307070280
:1027800093870702E31CD7FCB3872A0173900D10CF
:1027900003370A0023B00700630007022334F70061
:1027A0002330FA00B7170000B384F400E39864F50F
:1027B00003358100EFF05FAE2330FA0023B0FB0059
:1027C0006FF05FFE17150000130545AEEFF05FA830
:1027D00013053000EFF05FAC17150000130585B648
:1027E000EFF01FA76FF01FEB17150000130585AF63
:1027F000EFF01FA613053000EFF01FAAF32740F1FA
:10280000639A0718975700009387C77F130101ED5C
:1028100093D7C70023308112176800001308887E01
:10282000130405009397A700174500001305857D45
:10283000233411129356C5001357C80093E71700AD
:10284000973800009388087C1306F0FF233CF5FEC0
:102850009396A6001317A700B707002093E616006B
:102860001367170093D5C8001313F6039387F70C6B
:10287000233CF8FE23B0D8002330E500B3E7650021
:102880007390071873270018639EE7141356B60059
:102890009307F0019702000093824201F3925230B5
:1028A0007310063B7390073A739052301308F0BFD1
:1028B0001318580197E7FFFF9387078AB38707012B
:1028C00073905710F3270034B387070173900714F0
:1028D000B7B700009B87071073902730B7E7010058
:1028E0009B870760739007307350403017370000A4
:1028F000130747B09307083EB3060701B307F70075
:10290000B7080800177600002332D670173300008E
:10291000130343ED9776000023B6F66E9388F80311
:102920009307E0031308080113D61700B3861701B5
:10293000B347F600B30507019396C6009397570077
:102940002330D7002334B70093F70702130707019A
:10295000B367F600E31AE3FC1306001293050000C8
:10296000130501009737000023BA07E6EFF00FEFD9
:10297000B70700803304F4001305010023348110ED
:10298000EFD0CFF48330811203340112130101130D
:102990006780000013071000B7578004370608004F
:1029A000938767F91306C6FF1315F7019316E7031C
:1029B0006F00C0012F20070013D71700B3C7E7002F
:1029C0009397E703B3F7D700B3E7E70033F7C70000
:1029D00093F517003307A700E39E05FC03200700CB
:1029E0006FF09FFD171500001305C598EFF05F8687
:1029F00013053000EFF05F8A6780000013050000C8
:102A0000678000001305000067800000731030002D
:102A100093012000171500001305C55E072005006F
:102A200087204500072185008326C500531500C077
:102A3000F315100013061000631AD5726398C5725F
:102A400093013000171500001305C55C0720050031
:102A500087204500072185008326C500531500C047
:102A6000F3151000130600006312D5706390C57053
:102A700093014000171500001305C55A07200500F3
:102A800087204500072185008326C500531500C017
:102A9000F315100013061000631AD56C6398C56C0B
:102AA00093015000171500001305C55807200500B5
:102AB00087204500072185008326C500531500C0E7
:102AC000F3151000130610006312D56A6390C56AEF
:102AD00093016000171500001305C5560720050077
:102AE00087204500072185008326C500531500C0B7
:102AF000F315100013060000631AD5666398C566C7
:102B000093017000171500001305C5540720050038
:102B100087204500072185008326C500531500C086
:102B2000F3151000130610006312D5646390C5649A
:102B300093018000171500001305C55207200500FA
:102B400087204500072185008326C500531500C056
:102B5000F315100013060001631AD5606398C56071
:102B600093019000171500001305C55007200500BC
:102B700087204500072185008326C500531500C026
:102B8000F3151000130600016312D55E6390C55E55
:102B90009301C000171500001305C54E072005005E
:102BA00087204500072185008326C500531510C0E6
:102BB000F315100013060001631AD55A6398C55A1D
:102BC0009301D000171500001305C54C0720050020
:102BD00087204500072185008326C500531510C0B6
:102BE000F3151000130600016312D5586390C55801
:102BF0009301E000171500001305C54A07200500E2
:102C000087204500072185008326C500531510C085
:102C1000F315100013061000631AD5546398C554B9
:102C20009301F000171500001305C54807200500A3
:102C300087204500072185008326C500531510C055
:102C4000F3151000130610006312D5526390C5529D
:102C500093010001171500001305C5460720050064
:102C600087204500072185008326C500531510C025
:102C7000F315100013060000631AD54E6398C54E75
:102C800093011001171500001305C5440720050026
:102C900087204500072185008326C500531510C0F5
:102CA000F3151000130610006312D54C6390C54C49
:102CB00093012001171500001305C54207200500E8
:102CC00087204500072185008326C500531510C0C5
:102CD000F315100013060001631AD5486398C54820
:102CE00093013001171500001305C54007200500AA
:102CF00087204500072185008326C500531510C095
:102D0000F3151000130600006312D5466390C54604
:102D100093016001171500001305C53E072005004B
:102D200087204500072185008326C500531520C054
:102D3000F315100013061000631AD5426398C542BC
:102D400093017001171500001305C53C072005000D
:102D500087204500072185008326C500531520C024
:102D6000F3151000130600006312D5406390C540B0
:102D700093018001171500001305C53A07200500CF
:102D800087204500072185008326C500531520C0F4
:102D9000F315100013061000631AD53C6398C53C68
:102DA00093019001171500001305C5380720050091
:102DB00087204500072185008326C500531520C0C4
:102DC000F3151000130610006312D53A6390C53A4C
:102DD0009301A001171500001305C5360720050053
:102DE00087204500072185008326C500531520C094
:102DF000F315100013060000631AD5366398C53624
:102E00009301B001171500001305C5340720050014
:102E100087204500072185008326C500531520C063
:102E2000F3151000130610006312D5346390C534F7
:102E300093010002171500001305C5320720050095
:102E400087204500072185008326C500531530C023
:102E5000F315100013060001631AD5306398C530CE
:102E600093011002171500001305C5300720050057
:102E700087204500072185008326C500531530C0F3
:102E8000F3151000130600016312D52E6390C52EB2
:102E900093012002171500001305C52E0720050019
:102EA00087204500072185008326C500531530C0C3
:102EB000F315100013061000631AD52A6398C52A6B
:102EC00093013002171500001305C52C07200500DB
:102ED00087204500072185008326C500531530C093
:102EE000F3151000130610006312D5286390C5284F
:102EF00093014002171500001305C52A072005009D
:102F000087204500072185008326C500531530C062
:102F1000F315100013060000631AD5246398C52426
:102F200093015002171500001305C528072005005E
:102F300087204500072185008326C500531530C032
:102F4000F3151000130610006312D5226390C522FA
:102F500093016002171500001305C5260720050020
:102F600087204500072185008326C500531530C002
:102F7000F315100013060001631AD51E6398C51ED1
:102F80009301A002971000009380C02487A0000046
:102F9000D3F000C0B70300809B83F3FF6398701CDD
:102FA0009301C002971000009380C02287A0800088
:102FB000D3F000C0B7030080639A701A9301B00287
:102FC000971000009380002187A00000D3F020C05C
:102FD0009B03F0FF9393F3039383F3FF63987018BD
:102FE0009301D002971000009380C01E87A080003C
:102FF000D3F020C09B03F0FF9393F3036398701604
:1030000093014003971000009380C01C87A04000EC
:10301000D3F000C0B70300809B83F3FF6398701464
:1030200093016003971000009380C01A87A0C0002E
:10303000D3F000C0B70300809B83F3FF6398701246
:1030400093015003971000009380C01887A04000A0
:10305000D3F020C09B03F0FF9393F3039383F3FF1C
:103060006396701093017003971000009380801690
:1030700087A0C000D3F020C09B03F0FF9393F3031D
:103080009383F3FF6394700E9301E00397100000A5
:103090009380401487A00000D3F010C09303F0FF8A
:1030A0006396700C9301F0039710000093808012D8
:1030B00087A04000D3F010C09303F0FF6398700A1C
:1030C00093010004971000009380C01087A0800037
:1030D000D3F010C093030000639A700893011004AA
:1030E000971000009380000F87A0C000D3F010C09D
:1030F0009303F0FF639C7006930120049710000077
:103100009380400D87A00000D3F030C09303F0FF00
:10311000639E700493013004971000009380800B2D
:1031200087A04000D3F030C09303F0FF6390700499
:1031300093014004971000009380C00987A080008D
:10314000D3F030C0930300006392700293015004E7
:10315000971000009380000887A0C000D3F030C013
:103160009303F0FF63947000631A3000139511000D
:1031700063000500136515007300000013051000BF
:0831800073000000731000C091
:08318800010101010101010137
:10319000417373657274696F6E206661696C6564F2
:1031A0003A2061646472203E3D202831554C203C19
:1031B0003C203132292026262061646472203C2084
:1031C0003633202A202831554C203C3C20313229EE
:1031D0000A00000000000000417373657274696F9B
:1031E0006E206661696C65643A20212870745B33D7
:1031F0005D5B616464722F2831554C203C3C20316A
:1032000032295D20262030783038302920262620AB
:103210006361757365203D3D203078660A000000CB
:10322000417373657274696F6E206661696C656461
:103230003A206E6F64650A00417373657274696F3A
:103240006E206661696C65643A20757365725F6DA6
:10325000617070696E675B616464722F2831554CD0
:10326000203C3C203132295D2E61646472203D3D5A
:1032700020300A0000000000417373657274696FAA
:103280006E206661696C65643A202122696C6C6508
:1032900067616C20696E737472756374696F6E22F6
:1032A0000A00000000000000417373657274696FCA
:1032B0006E206661696C65643A2070745B335D5B97
:1032C000616464722F2831554C203C3C20313229F6
:1032D0005D20262030783034300A000000000000E5
:1032E000417373657274696F6E206661696C6564A1
:1032F0003A2070745B335D5B616464722F283155D2
:103300004C203C3C203132295D202620307830385A
:10331000300A000000000000417373657274696F29
:103320006E206661696C65643A2074662D3E657036
:103330006320252034203D3D20300A00000000009D
:10334000417373657274696F6E206661696C656440
:103350003A202122756E6578706563746564206516
:103360007863657074696F6E220A000000000000C7
:10337000417373657274696F6E206661696C656410
:103380003A202122756E737570706F7274656420B7
:0C33900073617470206D6F6465220A0088
:10400000CDCC8CBF0000000000000000FFFFFFFFD0
:10401000000080BF0000000000000000FFFFFFFF65
:10402000666666BF0000000000000000000000009F
:104030006666663F0000000000000000000000000F
:104040000000803F000000000000000001000000B0
:10405000CDCC8C3F000000000000000001000000FB
:104060005ED032CF000000000000000000000080A1
:104070005ED0324F0000000000000000FFFFFF7F15
:10408000000040C000000000000000000000000030
:10409000000080BF000000000000000000000000E1
:1040A000666666BF0000000000000000000000001F
:1040B0006666663F0000000000000000000000008F
:1040C0000000803F00000000000000000100000030
:1040D000CDCC8C3F0000000000000000010000007B
:1040E0005ED032CF000000000000000000000000A1
:1040F0005ED0324F0000000000000000005ED0B231
:10410000CDCC8CBF0000000000000000FFFFFFFFCF
:10411000000080BF0000000000000000FFFFFFFF64
:10412000666666BF0000000000000000000000009E
:104130006666663F0000000000000000000000000E
:104140000000803F000000000000000001000000AF
:10415000CDCC8C3F000000000000000001000000FA
:10416000000040C00000000000000000000000004F
:10417000000080BF00000000000000000000000000
:10418000666666BF0000000000000000000000003E
:104190006666663F000000000000000000000000AE
:1041A0000000803F0000000000000000010000004F
:1041B000CDCC8C3F0000000000000000010000009A
:1041C0005ED032CF000000000000000000000000C0
:1041D000FFFFFFFFFFFFFF7F000080FF0000807FE9
:1041E000FFFFFFFFFFFFFFFFFFFFFFFFFFFFFF7F5F
:1041F000000000000000F0FF000000000000F07F61
:040000058000000077
:00000001FF
